:020000040000FA
:020000000428D2
:08000800FF30A100FF30A2004F
:10001000FF30A300FF30A4000F30A50021108A118B
:100020000A12512005308A110A12282026148A113A
:100030000A124B2005308A110A12282026108A1134
:100040000A124B208A110A1212288A110A12252834
:10005000A7002708A8006430A9000A308A110A12F4
:100060003128AA00FF30AB002908AD002808AC00F9
:1000700077308A110A122B0703183B288A110A12BB
:10008000AC0B38288A110A12AD0B36288A110A12D5
:10009000AA0B342808008A110A124E282608850067
:0E00A00008008A110A12542821086500080081
:02400E00F23F7F
:00000001FF
